 timerinfo001

 Timestamp is 5b6be727 (reproducible build file hash)

 Preferred load address is 0000000180000000

 Start         Length     Name                   Class
 0001:00000000 000037d0H .text$mn                CODE
 0001:000037d0 00000036H .text$mn$00             CODE
 0001:00003806 00000092H .text$x                 CODE
 0002:00000000 000001c8H .idata$5                DATA
 0002:000001c8 00000038H .00cfg                  DATA
 0002:00000200 00000008H .CRT$XCA                DATA
 0002:00000208 00000008H .CRT$XCZ                DATA
 0002:00000210 00000008H .CRT$XIA                DATA
 0002:00000218 00000008H .CRT$XIC                DATA
 0002:00000220 00000008H .CRT$XIZ                DATA
 0002:00000228 00000008H .CRT$XLA                DATA
 0002:00000230 00000008H .CRT$XLZ                DATA
 0002:00000238 00000008H .CRT$XPA                DATA
 0002:00000240 00000008H .CRT$XPZ                DATA
 0002:00000248 00000008H .CRT$XTA                DATA
 0002:00000250 00000010H .CRT$XTZ                DATA
 0002:00000258 00000000H .gehcont$y              DATA
 0002:00000258 00000000H .gfids$y                DATA
 0002:00000260 00002220H .rdata                  DATA
 0002:00002480 00000000H .rdata$CastGuardVftablesA DATA
 0002:00002480 00000000H .rdata$CastGuardVftablesC DATA
 0002:00002480 00000028H .rdata$T                DATA
 0002:000024a8 000000e4H .rdata$voltmd           DATA
 0002:0000258c 0000031cH .rdata$zzzdbg           DATA
 0002:000028a8 00000008H .rtc$IAA                DATA
 0002:000028b0 00000008H .rtc$IZZ                DATA
 0002:000028b8 00000008H .rtc$TAA                DATA
 0002:000028c0 00000008H .rtc$TZZ                DATA
 0002:000028c8 00000004H .tls                    DATA
 0002:000028cc 00000004H .tls$                   DATA
 0002:000028d0 00000008H .tls$ZZZ                DATA
 0002:000028d8 00000398H .xdata                  DATA
 0002:00002c70 00000398H .edata                  DATA
 0002:00003008 0000008cH .idata$2                DATA
 0002:00003094 00000014H .idata$3                DATA
 0002:000030a8 000001c8H .idata$4                DATA
 0002:00003270 00000486H .idata$6                DATA
 0003:00000000 00000080H .data                   DATA
 0003:00000080 0001b258H .bss                    DATA
 0004:00000000 000003f0H .pdata                  DATA

  Address         Publics by Value              Rva+Base               Lib:Object

 0000:00000000       __AbsoluteZero             0000000000000000     <absolute>
 0000:00000000       ___safe_se_handler_count   0000000000000000     <absolute>
 0000:00000000       ___safe_se_handler_table   0000000000000000     <absolute>
 0000:00000000       __arm64x_extra_rfe_table   0000000000000000     <absolute>
 0000:00000000       __arm64x_extra_rfe_table_size 0000000000000000     <absolute>
 0000:00000000       __arm64x_native_entrypoint 0000000000000000     <absolute>
 0000:00000000       __arm64x_redirection_metadata 0000000000000000     <absolute>
 0000:00000000       __arm64x_redirection_metadata_count 0000000000000000     <absolute>
 0000:00000000       __dynamic_value_reloc_table 0000000000000000     <absolute>
 0000:00000000       __enclave_config           0000000000000000     <absolute>
 0000:00000000       __guard_check_icall_a64n_fptr 0000000000000000     <absolute>
 0000:00000000       __guard_eh_cont_count      0000000000000000     <absolute>
 0000:00000000       __guard_eh_cont_table      0000000000000000     <absolute>
 0000:00000000       __guard_fids_count         0000000000000000     <absolute>
 0000:00000000       __guard_fids_table         0000000000000000     <absolute>
 0000:00000000       __guard_iat_count          0000000000000000     <absolute>
 0000:00000000       __guard_iat_table          0000000000000000     <absolute>
 0000:00000000       __guard_longjmp_count      0000000000000000     <absolute>
 0000:00000000       __guard_longjmp_table      0000000000000000     <absolute>
 0000:00000000       __hybrid_auxiliary_iat     0000000000000000     <absolute>
 0000:00000000       __hybrid_auxiliary_iat_copy 0000000000000000     <absolute>
 0000:00000000       __hybrid_code_map          0000000000000000     <absolute>
 0000:00000000       __hybrid_code_map_count    0000000000000000     <absolute>
 0000:00000000       __x64_code_ranges_to_entry_points 0000000000000000     <absolute>
 0000:00000000       __x64_code_ranges_to_entry_points_count 0000000000000000     <absolute>
 0000:00000100       __guard_flags              0000000000000100     <absolute>
 0000:00000000       __ImageBase                0000000180000000     <linker-defined>
 0001:00000000       ?NewObject@JNIEnv_@@QEAAPEAV_jobject@@PEAV_jclass@@PEAU_jmethodID@@ZZ 0000000180001000 f i libtimerinfo001.obj
 0001:00000024       ?SetEventNotificationMode@_jvmtiEnv@@QEAA?AW4jvmtiError@@W4jvmtiEventMode@@W4jvmtiEvent@@PEAV_jobject@@ZZ 0000000180001024 f i libtimerinfo001.obj
 0001:0000002c       ?TranslateError@@YAPEBDW4jvmtiError@@@Z 000000018000102c f   libtimerinfo001.obj
 0001:000002e4       ?julong_to_string@@YAPEAD_KPEAD@Z 00000001800012e4 f   libtimerinfo001.obj
 0001:00000374       ?nsk_jni_check_exception@@YAHPEAUJNIEnv_@@QEBDH@Z 0000000180001374 f   libtimerinfo001.obj
 0001:000004b8       ?nsk_jni_lverify@@YAHHPEAUJNIEnv_@@HQEBDH1ZZ 00000001800014b8 f   libtimerinfo001.obj
 0001:00000558       Agent_Initialize           0000000180001558 f   libtimerinfo001.obj
 0001:000007d0       Agent_OnAttach             00000001800017d0 f   libtimerinfo001.obj
 0001:000007d0       Agent_OnLoad               00000001800017d0 f   libtimerinfo001.obj
 0001:000007d8       Java_nsk_jvmti_unit_FollowReferences_FollowRefObjects_addRefToVerify 00000001800017d8 f   libtimerinfo001.obj
 0001:00000994       Java_nsk_jvmti_unit_FollowReferences_FollowRefObjects_getTag 0000000180001994 f   libtimerinfo001.obj
 0001:00000a50       Java_nsk_jvmti_unit_FollowReferences_FollowRefObjects_resetRefsToVerify 0000000180001a50 f   libtimerinfo001.obj
 0001:00000a58       Java_nsk_jvmti_unit_FollowReferences_FollowRefObjects_resetTags 0000000180001a58 f   libtimerinfo001.obj
 0001:00000a9c       Java_nsk_jvmti_unit_FollowReferences_FollowRefObjects_setTag 0000000180001a9c f   libtimerinfo001.obj
 0001:00000ce8       Java_nsk_share_jvmti_ArgumentHandler_getAgentOptionsString 0000000180001ce8 f   libtimerinfo001.obj
 0001:00000d94       Java_nsk_share_jvmti_DebugeeClass_checkStatus 0000000180001d94 f   libtimerinfo001.obj
 0001:00000e1c       Java_nsk_share_jvmti_DebugeeClass_resetAgentData 0000000180001e1c f   libtimerinfo001.obj
 0001:00000e7c       Java_nsk_share_jvmti_RedefineAgent_agentStatus 0000000180001e7c f   libtimerinfo001.obj
 0001:00000e88       Java_nsk_share_jvmti_RedefineAgent_isRedefined 0000000180001e88 f   libtimerinfo001.obj
 0001:00000e94       Java_nsk_share_jvmti_RedefineAgent_redefineAttempted 0000000180001e94 f   libtimerinfo001.obj
 0001:00000ea0       MA_checkStatus             0000000180001ea0 f   libtimerinfo001.obj
 0001:00000f44       __local_stdio_printf_options 0000000180001f44 f i libtimerinfo001.obj
 0001:000011c8       callbackVMDeath            00000001800021c8 f   libtimerinfo001.obj
 0001:000012c4       callbackVMInit             00000001800022c4 f   libtimerinfo001.obj
 0001:00001720       exitOnError                0000000180002720 f   libtimerinfo001.obj
 0001:000017d4       fprintf                    00000001800027d4 f i libtimerinfo001.obj
 0001:00001818       nsk_complain               0000000180002818 f   libtimerinfo001.obj
 0001:00001844       nsk_jvmti_createJVMTIEnv   0000000180002844 f   libtimerinfo001.obj
 0001:00001974       nsk_jvmti_enableEvents     0000000180002974 f   libtimerinfo001.obj
 0001:00001a50       nsk_jvmti_lverify          0000000180002a50 f   libtimerinfo001.obj
 0001:00001b40       nsk_jvmti_parseOptions     0000000180002b40 f   libtimerinfo001.obj
 0001:00001d90       nsk_jvmti_resetAgentData   0000000180002d90 f   libtimerinfo001.obj
 0001:00001e04       nsk_jvmti_resumeSync       0000000180002e04 f   libtimerinfo001.obj
 0001:00001ea8       nsk_jvmti_waitForSync      0000000180002ea8 f   libtimerinfo001.obj
 0001:00001fac       nsk_lcomplain              0000000180002fac f   libtimerinfo001.obj
 0001:00001fcc       nsk_ldisplay               0000000180002fcc f   libtimerinfo001.obj
 0001:00001fec       nsk_ltrace                 0000000180002fec f   libtimerinfo001.obj
 0001:0000200c       nsk_lvcomplain             000000018000300c f   libtimerinfo001.obj
 0001:000021c4       nsk_lvdisplay              00000001800031c4 f   libtimerinfo001.obj
 0001:00002210       nsk_lverify                0000000180003210 f   libtimerinfo001.obj
 0001:0000226c       nsk_lvtrace                000000018000326c f   libtimerinfo001.obj
 0001:000022cc       nsk_printf                 00000001800032cc f   libtimerinfo001.obj
 0001:000022f4       nsk_vprintf                00000001800032f4 f   libtimerinfo001.obj
 0001:000023a8       printf                     00000001800033a8 f i libtimerinfo001.obj
 0001:000028a8       __raise_securityfailure    00000001800038a8 f   MSVCRT:gs_report.obj
 0001:000028dc       __report_gsfailure         00000001800038dc f   MSVCRT:gs_report.obj
 0001:00002b1c       __GSHandlerCheck           0000000180003b1c f   MSVCRT:gshandler.obj
 0001:00002b3c       __GSHandlerCheckCommon     0000000180003b3c f   MSVCRT:gshandler.obj
 0001:00002bb0       __security_check_cookie    0000000180003bb0 f   MSVCRT:amdsecgs.obj
 0001:00002ef0       _DllMainCRTStartup         0000000180003ef0 f   MSVCRT:dll_dllmain.obj
 0001:00002f30       __scrt_acquire_startup_lock 0000000180003f30 f   MSVCRT:utility.obj
 0001:00002f6c       __scrt_dllmain_after_initialize_c 0000000180003f6c f   MSVCRT:utility.obj
 0001:00002fa0       __scrt_dllmain_before_initialize_c 0000000180003fa0 f   MSVCRT:utility.obj
 0001:00002fb8       __scrt_dllmain_crt_thread_attach 0000000180003fb8 f   MSVCRT:utility.obj
 0001:00002fe0       __scrt_dllmain_crt_thread_detach 0000000180003fe0 f   MSVCRT:utility.obj
 0001:00002ff8       __scrt_dllmain_exception_filter 0000000180003ff8 f   MSVCRT:utility.obj
 0001:00003058       __scrt_dllmain_uninitialize_c 0000000180004058 f   MSVCRT:utility.obj
 0001:00003088       __scrt_dllmain_uninitialize_critical 0000000180004088 f   MSVCRT:utility.obj
 0001:0000309c       __scrt_initialize_crt      000000018000409c f   MSVCRT:utility.obj
 0001:000030e8       __scrt_initialize_onexit_tables 00000001800040e8 f   MSVCRT:utility.obj
 0001:00003174       __scrt_is_nonwritable_in_current_image 0000000180004174 f   MSVCRT:utility.obj
 0001:0000320c       __scrt_release_startup_lock 000000018000420c f   MSVCRT:utility.obj
 0001:00003230       __scrt_uninitialize_crt    0000000180004230 f   MSVCRT:utility.obj
 0001:0000325c       _onexit                    000000018000425c f   MSVCRT:utility.obj
 0001:00003298       atexit                     0000000180004298 f   MSVCRT:utility.obj
 0001:000032b0       __crt_debugger_hook        00000001800042b0 f   MSVCRT:utility_desktop.obj
 0001:000032b8       __scrt_fastfail            00000001800042b8 f   MSVCRT:utility_desktop.obj
 0001:00003404       _guard_check_icall_nop     0000000180004404 f i MSVCRT:guard_support.obj
 0001:00003408       __security_init_cookie     0000000180004408 f   MSVCRT:gs_support.obj
 0001:000034b4       DllMain                    00000001800044b4 f   MSVCRT:dll_dllmain_stub.obj
 0001:000034d8       ?__scrt_initialize_type_info@@YAXXZ 00000001800044d8 f   MSVCRT:tncleanup.obj
 0001:000034e8       ?__scrt_uninitialize_type_info@@YAXXZ 00000001800044e8 f   MSVCRT:tncleanup.obj
 0001:000034f4       __local_stdio_scanf_options 00000001800044f4 f i MSVCRT:default_local_stdio_options.obj
 0001:000034fc       __scrt_initialize_default_local_stdio_options 00000001800044fc f   MSVCRT:default_local_stdio_options.obj
 0001:00003518       __scrt_get_dyn_tls_init_callback 0000000180004518 f   MSVCRT:dyn_tls_init.obj
 0001:00003520       _RTC_Initialize            0000000180004520 f   MSVCRT:initsect.obj
 0001:0000355c       _RTC_Terminate             000000018000455c f   MSVCRT:initsect.obj
 0001:00003598       __isa_available_init       0000000180004598 f   MSVCRT:cpu_disp.obj
 0001:00003744       _get_startup_argv_mode     0000000180004744 f   MSVCRT:argv_mode.obj
 0001:0000374c       __scrt_is_ucrt_dll_in_use  000000018000474c f   MSVCRT:ucrt_detection.obj
 0001:00003760       memcpy                     0000000180004760 f   vcruntime:VCRUNTIME140.dll
 0001:00003766       memset                     0000000180004766 f   vcruntime:VCRUNTIME140.dll
 0001:0000376c       strchr                     000000018000476c f   vcruntime:VCRUNTIME140.dll
 0001:00003772       __C_specific_handler       0000000180004772 f   vcruntime:VCRUNTIME140.dll
 0001:00003778       __std_type_info_destroy_list 0000000180004778 f   vcruntime:VCRUNTIME140.dll
 0001:0000377e       strcmp                     000000018000477e f   ucrt:api-ms-win-crt-string-l1-1-0.dll
 0001:00003784       strlen                     0000000180004784 f   ucrt:api-ms-win-crt-string-l1-1-0.dll
 0001:0000378a       _initterm                  000000018000478a f   ucrt:api-ms-win-crt-runtime-l1-1-0.dll
 0001:00003790       _initterm_e                0000000180004790 f   ucrt:api-ms-win-crt-runtime-l1-1-0.dll
 0001:00003796       _seh_filter_dll            0000000180004796 f   ucrt:api-ms-win-crt-runtime-l1-1-0.dll
 0001:0000379c       _configure_narrow_argv     000000018000479c f   ucrt:api-ms-win-crt-runtime-l1-1-0.dll
 0001:000037a2       _initialize_narrow_environment 00000001800047a2 f   ucrt:api-ms-win-crt-runtime-l1-1-0.dll
 0001:000037a8       _initialize_onexit_table   00000001800047a8 f   ucrt:api-ms-win-crt-runtime-l1-1-0.dll
 0001:000037ae       _register_onexit_function  00000001800047ae f   ucrt:api-ms-win-crt-runtime-l1-1-0.dll
 0001:000037b4       _execute_onexit_table      00000001800047b4 f   ucrt:api-ms-win-crt-runtime-l1-1-0.dll
 0001:000037ba       _crt_atexit                00000001800047ba f   ucrt:api-ms-win-crt-runtime-l1-1-0.dll
 0001:000037c0       _cexit                     00000001800047c0 f   ucrt:api-ms-win-crt-runtime-l1-1-0.dll
 0001:000037c8       __acrt_initialize          00000001800047c8 f   MSVCRT:ucrt_stubs.obj
 0001:000037c8       __acrt_thread_attach       00000001800047c8 f   MSVCRT:ucrt_stubs.obj
 0001:000037c8       __acrt_thread_detach       00000001800047c8 f   MSVCRT:ucrt_stubs.obj
 0001:000037c8       __acrt_uninitialize        00000001800047c8 f   MSVCRT:ucrt_stubs.obj
 0001:000037c8       __acrt_uninitialize_critical 00000001800047c8 f   MSVCRT:ucrt_stubs.obj
 0001:000037c8       __scrt_stub_for_acrt_initialize 00000001800047c8 f   MSVCRT:ucrt_stubs.obj
 0001:000037c8       __scrt_stub_for_acrt_thread_attach 00000001800047c8 f   MSVCRT:ucrt_stubs.obj
 0001:000037c8       __scrt_stub_for_acrt_thread_detach 00000001800047c8 f   MSVCRT:ucrt_stubs.obj
 0001:000037c8       __scrt_stub_for_acrt_uninitialize 00000001800047c8 f   MSVCRT:ucrt_stubs.obj
 0001:000037c8       __scrt_stub_for_acrt_uninitialize_critical 00000001800047c8 f   MSVCRT:ucrt_stubs.obj
 0001:000037c8       __vcrt_initialize          00000001800047c8 f   MSVCRT:ucrt_stubs.obj
 0001:000037c8       __vcrt_thread_attach       00000001800047c8 f   MSVCRT:ucrt_stubs.obj
 0001:000037c8       __vcrt_thread_detach       00000001800047c8 f   MSVCRT:ucrt_stubs.obj
 0001:000037c8       __vcrt_uninitialize        00000001800047c8 f   MSVCRT:ucrt_stubs.obj
 0001:000037c8       __vcrt_uninitialize_critical 00000001800047c8 f   MSVCRT:ucrt_stubs.obj
 0001:000037cc       __scrt_stub_for_is_c_termination_complete 00000001800047cc f   MSVCRT:ucrt_stubs.obj
 0001:000037cc       _is_c_termination_complete 00000001800047cc f   MSVCRT:ucrt_stubs.obj
 0001:000037e0       _guard_dispatch_icall_nop  00000001800047e0 f   MSVCRT:guard_dispatch.obj
 0001:00003800       _guard_xfg_dispatch_icall_nop 0000000180004800 f   MSVCRT:guard_xfg_dispatch.obj
 0002:00000000       __imp_RtlCaptureContext    0000000180005000     kernel32:KERNEL32.dll
 0002:00000008       __imp_RtlLookupFunctionEntry 0000000180005008     kernel32:KERNEL32.dll
 0002:00000010       __imp_RtlVirtualUnwind     0000000180005010     kernel32:KERNEL32.dll
 0002:00000018       __imp_UnhandledExceptionFilter 0000000180005018     kernel32:KERNEL32.dll
 0002:00000020       __imp_SetUnhandledExceptionFilter 0000000180005020     kernel32:KERNEL32.dll
 0002:00000028       __imp_GetCurrentProcess    0000000180005028     kernel32:KERNEL32.dll
 0002:00000030       __imp_TerminateProcess     0000000180005030     kernel32:KERNEL32.dll
 0002:00000038       __imp_IsProcessorFeaturePresent 0000000180005038     kernel32:KERNEL32.dll
 0002:00000040       __imp_CloseHandle          0000000180005040     kernel32:KERNEL32.dll
 0002:00000048       __imp_InitializeCriticalSectionAndSpinCount 0000000180005048     kernel32:KERNEL32.dll
 0002:00000050       __imp_DeleteCriticalSection 0000000180005050     kernel32:KERNEL32.dll
 0002:00000058       __imp_CreateEventW         0000000180005058     kernel32:KERNEL32.dll
 0002:00000060       __imp_GetModuleHandleW     0000000180005060     kernel32:KERNEL32.dll
 0002:00000068       __imp_GetProcAddress       0000000180005068     kernel32:KERNEL32.dll
 0002:00000070       __imp_IsDebuggerPresent    0000000180005070     kernel32:KERNEL32.dll
 0002:00000078       __imp_QueryPerformanceCounter 0000000180005078     kernel32:KERNEL32.dll
 0002:00000080       __imp_GetCurrentProcessId  0000000180005080     kernel32:KERNEL32.dll
 0002:00000088       __imp_GetCurrentThreadId   0000000180005088     kernel32:KERNEL32.dll
 0002:00000090       __imp_GetSystemTimeAsFileTime 0000000180005090     kernel32:KERNEL32.dll
 0002:00000098       __imp_DisableThreadLibraryCalls 0000000180005098     kernel32:KERNEL32.dll
 0002:000000a0       __imp_InitializeSListHead  00000001800050a0     kernel32:KERNEL32.dll
 0002:000000a8       \177KERNEL32_NULL_THUNK_DATA 00000001800050a8     kernel32:KERNEL32.dll
 0002:000000b0       __imp_memcpy               00000001800050b0     vcruntime:VCRUNTIME140.dll
 0002:000000b8       __imp_memset               00000001800050b8     vcruntime:VCRUNTIME140.dll
 0002:000000c0       __imp_strchr               00000001800050c0     vcruntime:VCRUNTIME140.dll
 0002:000000c8       __imp___C_specific_handler 00000001800050c8     vcruntime:VCRUNTIME140.dll
 0002:000000d0       __imp___std_type_info_destroy_list 00000001800050d0     vcruntime:VCRUNTIME140.dll
 0002:000000d8       \177VCRUNTIME140_NULL_THUNK_DATA 00000001800050d8     vcruntime:VCRUNTIME140.dll
 0002:000000e0       __imp_strtol               00000001800050e0     ucrt:api-ms-win-crt-convert-l1-1-0.dll
 0002:000000e8       \177api-ms-win-crt-convert-l1-1-0_NULL_THUNK_DATA 00000001800050e8     ucrt:api-ms-win-crt-convert-l1-1-0.dll
 0002:000000f0       __imp_malloc               00000001800050f0     ucrt:api-ms-win-crt-heap-l1-1-0.dll
 0002:000000f8       __imp_free                 00000001800050f8     ucrt:api-ms-win-crt-heap-l1-1-0.dll
 0002:00000100       \177api-ms-win-crt-heap-l1-1-0_NULL_THUNK_DATA 0000000180005100     ucrt:api-ms-win-crt-heap-l1-1-0.dll
 0002:00000108       __imp__errno               0000000180005108     ucrt:api-ms-win-crt-runtime-l1-1-0.dll
 0002:00000110       __imp_exit                 0000000180005110     ucrt:api-ms-win-crt-runtime-l1-1-0.dll
 0002:00000118       __imp__cexit               0000000180005118     ucrt:api-ms-win-crt-runtime-l1-1-0.dll
 0002:00000120       __imp__crt_atexit          0000000180005120     ucrt:api-ms-win-crt-runtime-l1-1-0.dll
 0002:00000128       __imp__execute_onexit_table 0000000180005128     ucrt:api-ms-win-crt-runtime-l1-1-0.dll
 0002:00000130       __imp__register_onexit_function 0000000180005130     ucrt:api-ms-win-crt-runtime-l1-1-0.dll
 0002:00000138       __imp__initialize_onexit_table 0000000180005138     ucrt:api-ms-win-crt-runtime-l1-1-0.dll
 0002:00000140       __imp__initialize_narrow_environment 0000000180005140     ucrt:api-ms-win-crt-runtime-l1-1-0.dll
 0002:00000148       __imp__configure_narrow_argv 0000000180005148     ucrt:api-ms-win-crt-runtime-l1-1-0.dll
 0002:00000150       __imp__seh_filter_dll      0000000180005150     ucrt:api-ms-win-crt-runtime-l1-1-0.dll
 0002:00000158       __imp__initterm_e          0000000180005158     ucrt:api-ms-win-crt-runtime-l1-1-0.dll
 0002:00000160       __imp__initterm            0000000180005160     ucrt:api-ms-win-crt-runtime-l1-1-0.dll
 0002:00000168       \177api-ms-win-crt-runtime-l1-1-0_NULL_THUNK_DATA 0000000180005168     ucrt:api-ms-win-crt-runtime-l1-1-0.dll
 0002:00000170       __imp___acrt_iob_func      0000000180005170     ucrt:api-ms-win-crt-stdio-l1-1-0.dll
 0002:00000178       __imp_fflush               0000000180005178     ucrt:api-ms-win-crt-stdio-l1-1-0.dll
 0002:00000180       __imp___stdio_common_vsprintf 0000000180005180     ucrt:api-ms-win-crt-stdio-l1-1-0.dll
 0002:00000188       __imp___stdio_common_vfprintf 0000000180005188     ucrt:api-ms-win-crt-stdio-l1-1-0.dll
 0002:00000190       \177api-ms-win-crt-stdio-l1-1-0_NULL_THUNK_DATA 0000000180005190     ucrt:api-ms-win-crt-stdio-l1-1-0.dll
 0002:00000198       __imp_strcmp               0000000180005198     ucrt:api-ms-win-crt-string-l1-1-0.dll
 0002:000001a0       __imp__strdup              00000001800051a0     ucrt:api-ms-win-crt-string-l1-1-0.dll
 0002:000001a0       __imp_strdup               00000001800051a0     ucrt:api-ms-win-crt-string-l1-1-0.dll
 0002:000001a8       __imp_strlen               00000001800051a8     ucrt:api-ms-win-crt-string-l1-1-0.dll
 0002:000001b0       __imp_strpbrk              00000001800051b0     ucrt:api-ms-win-crt-string-l1-1-0.dll
 0002:000001b8       __imp_strncpy              00000001800051b8     ucrt:api-ms-win-crt-string-l1-1-0.dll
 0002:000001c0       \177api-ms-win-crt-string-l1-1-0_NULL_THUNK_DATA 00000001800051c0     ucrt:api-ms-win-crt-string-l1-1-0.dll
 0002:000001c8       __guard_check_icall_fptr   00000001800051c8     MSVCRT:guard_support.obj
 0002:000001d0       __guard_xfg_check_icall_fptr 00000001800051d0     MSVCRT:guard_support.obj
 0002:000001d8       __guard_dispatch_icall_fptr 00000001800051d8     MSVCRT:guard_support.obj
 0002:000001e0       __guard_xfg_dispatch_icall_fptr 00000001800051e0     MSVCRT:guard_support.obj
 0002:000001e8       __guard_xfg_table_dispatch_icall_fptr 00000001800051e8     MSVCRT:guard_support.obj
 0002:000001f0       __castguard_check_failure_os_handled_fptr 00000001800051f0     MSVCRT:guard_support.obj
 0002:000001f8       __guard_memcpy_fptr        00000001800051f8     vcruntime:softmemtag.obj
 0002:00000200       __xc_a                     0000000180005200     MSVCRT:initializers.obj
 0002:00000208       __xc_z                     0000000180005208     MSVCRT:initializers.obj
 0002:00000210       __xi_a                     0000000180005210     MSVCRT:initializers.obj
 0002:00000220       __xi_z                     0000000180005220     MSVCRT:initializers.obj
 0002:00000228       __xl_a                     0000000180005228     MSVCRT:tlssup.obj
 0002:00000230       __xl_z                     0000000180005230     MSVCRT:tlssup.obj
 0002:00000238       __xp_a                     0000000180005238     MSVCRT:initializers.obj
 0002:00000240       __xp_z                     0000000180005240     MSVCRT:initializers.obj
 0002:00000248       __xt_a                     0000000180005248     MSVCRT:initializers.obj
 0002:00000250       __xt_z                     0000000180005250     MSVCRT:initializers.obj
 0002:00000260       g_refKindStr               0000000180005260     libtimerinfo001.obj
 0002:00000410       ??_C@_09BPLDFGCI@unknown_0@ 0000000180005410     libtimerinfo001.obj
 0002:00000420       ??_C@_0BL@FPNMECJD@JVMTI_HEAP_REFERENCE_CLASS@ 0000000180005420     libtimerinfo001.obj
 0002:00000440       ??_C@_0BL@FKGKKLNM@JVMTI_HEAP_REFERENCE_FIELD@ 0000000180005440     libtimerinfo001.obj
 0002:00000460       ??_C@_0CD@CAEHCFJF@JVMTI_HEAP_REFERENCE_ARRAY_ELEM@ 0000000180005460     libtimerinfo001.obj
 0002:00000488       ??_C@_0CC@DNEBMCNK@JVMTI_HEAP_REFERENCE_CLASS_LOAD@ 0000000180005488     libtimerinfo001.obj
 0002:000004b0       ??_C@_0BN@CJMIPEBB@JVMTI_HEAP_REFERENCE_SIGNERS@ 00000001800054b0     libtimerinfo001.obj
 0002:000004d0       ??_C@_0CH@HBOIDPEB@JVMTI_HEAP_REFERENCE_PROTECTION@ 00000001800054d0     libtimerinfo001.obj
 0002:000004f8       ??_C@_0BP@MDKGDGKL@JVMTI_HEAP_REFERENCE_INTERFACE@ 00000001800054f8     libtimerinfo001.obj
 0002:00000518       ??_C@_0CC@JJMIHNJH@JVMTI_HEAP_REFERENCE_STATIC_FIE@ 0000000180005518     libtimerinfo001.obj
 0002:00000540       ??_C@_0CD@IDHEEGID@JVMTI_HEAP_REFERENCE_CONSTANT_P@ 0000000180005540     libtimerinfo001.obj
 0002:00000568       ??_C@_0CA@EFFCHNG@JVMTI_HEAP_REFERENCE_SUPERCLASS@ 0000000180005568     libtimerinfo001.obj
 0002:00000588       ??_C@_0L@PCDFHGCJ@unknown_11@ 0000000180005588     libtimerinfo001.obj
 0002:00000598       ??_C@_0L@NJBICFOK@unknown_12@ 0000000180005598     libtimerinfo001.obj
 0002:000005a8       ??_C@_0L@MAADBEKL@unknown_13@ 00000001800055a8     libtimerinfo001.obj
 0002:000005b8       ??_C@_0L@IPECICGM@unknown_14@ 00000001800055b8     libtimerinfo001.obj
 0002:000005c8       ??_C@_0L@JGFJLDCN@unknown_15@ 00000001800055c8     libtimerinfo001.obj
 0002:000005d8       ??_C@_0L@LNHEOAOO@unknown_16@ 00000001800055d8     libtimerinfo001.obj
 0002:000005e8       ??_C@_0L@KEGPNBKP@unknown_17@ 00000001800055e8     libtimerinfo001.obj
 0002:000005f8       ??_C@_0L@CDPHMNGA@unknown_18@ 00000001800055f8     libtimerinfo001.obj
 0002:00000608       ??_C@_0L@DKOMPMCB@unknown_19@ 0000000180005608     libtimerinfo001.obj
 0002:00000618       ??_C@_0L@OJGIPJDB@unknown_20@ 0000000180005618     libtimerinfo001.obj
 0002:00000628       ??_C@_0CA@KAOFNDEM@JVMTI_HEAP_REFERENCE_JNI_GLOBAL@ 0000000180005628     libtimerinfo001.obj
 0002:00000648       ??_C@_0CC@HPFAJBK@JVMTI_HEAP_REFERENCE_SYSTEM_CLA@ 0000000180005648     libtimerinfo001.obj
 0002:00000670       ??_C@_0BN@FDEGFOHC@JVMTI_HEAP_REFERENCE_MONITOR@ 0000000180005670     libtimerinfo001.obj
 0002:00000690       ??_C@_0CB@HKIBCMAJ@JVMTI_HEAP_REFERENCE_STACK_LOCA@ 0000000180005690     libtimerinfo001.obj
 0002:000006b8       ??_C@_0BP@EAACMMOE@JVMTI_HEAP_REFERENCE_JNI_LOCAL@ 00000001800056b8     libtimerinfo001.obj
 0002:000006d8       ??_C@_0BM@IJDEOGOE@JVMTI_HEAP_REFERENCE_THREAD@ 00000001800056d8     libtimerinfo001.obj
 0002:000006f8       ??_C@_0BL@EDGPPKC@JVMTI_HEAP_REFERENCE_OTHER@ 00000001800056f8     libtimerinfo001.obj
 0002:00000714       ??_C@_04BCJPDBDA@Code@     0000000180005714     libtimerinfo001.obj
 0002:00000720       ??_C@_0BA@OCLMCFKC@LineNumberTable@ 0000000180005720     libtimerinfo001.obj
 0002:00000730       ??_C@_0BD@CPAEPILC@LocalVariableTable@ 0000000180005730     libtimerinfo001.obj
 0002:00000748       ??_C@_0BH@NMBDNHBD@LocalVariableTypeTable@ 0000000180005748     libtimerinfo001.obj
 0002:00000760       ??_C@_0O@HIHEEDNJ@StackMapTable@ 0000000180005760     libtimerinfo001.obj
 0002:00000770       ??_C@_0L@HCDIAMJG@?9?5?$CFs?0?5?$CFd?3?5@ 0000000180005770     libtimerinfo001.obj
 0002:00000780       ??_C@_0JI@HLPECLFI@?$CD?5?4?4?4?6?$CD?5ERROR?3?5too?5many?5complai@ 0000000180005780     libtimerinfo001.obj
 0002:00000820       ??_C@_0ED@JNEKCCOB@The?5following?5fake?5exception?5st@ 0000000180005820     libtimerinfo001.obj
 0002:00000868       ??_C@_0CN@FCNMDFBH@nsk?4share?4Fake_Exception_for_RU@ 0000000180005868     libtimerinfo001.obj
 0002:00000898       ??_C@_08PGFFNAEI@?$CI?$CFs?3?$CFd?$CJ?5@ 0000000180005898     libtimerinfo001.obj
 0002:000008a8       ??_C@_0DP@IENMAEGI@s?2test?2hotspot?2jtreg?2vmTestbase@ 00000001800058a8     libtimerinfo001.obj
 0002:000008e8       ??_C@_0BL@NDJLFFJB@?7at?5nsk_lvcomplain?$CI?$CFs?3?$CFd?$CJ?6@ 00000001800058e8     libtimerinfo001.obj
 0002:00000908       ??_C@_0BC@JOOKAFKF@?$CD?5ERROR?3?5?$CFs?0?5?$CFd?3?5@ 0000000180005908     libtimerinfo001.obj
 0002:00000920       ??_C@_09KJEAHMEH@?$CD?5ERROR?3?5@ 0000000180005920     libtimerinfo001.obj
 0002:0000092c       ??_C@_02GPIOPFAK@?$DO?$DO@ 000000018000592c     libtimerinfo001.obj
 0002:00000930       ??_C@_02FODMEDOG@?$DM?$DM@ 0000000180005930     libtimerinfo001.obj
 0002:00000934       ??_C@_02DJGKEECL@?4?4@     0000000180005934     libtimerinfo001.obj
 0002:00000938       ??_C@_0O@CJPGJOAF@?9?5?$CFs?0?5?$CFd?3?5?$CFs?5@ 0000000180005938     libtimerinfo001.obj
 0002:00000948       ??_C@_0CB@IAKPDOIC@?$CD?5?5?5verified?5assertion?5is?5FALSE@ 0000000180005948     libtimerinfo001.obj
 0002:00000970       ??_C@_0CO@LGONDEPD@stdout?3?5fflush?5failed?5?9?5err?$DN?$CFd?5@ 0000000180005970     libtimerinfo001.obj
 0002:000009a0       ??_C@_0CO@KBGKJPBD@stderr?3?5fflush?5failed?5?9?5err?$DN?$CFd?5@ 00000001800059a0     libtimerinfo001.obj
 0002:000009d0       ??_C@_0BB@JCNMKLLK@JVMTI_ERROR_NONE@ 00000001800059d0     libtimerinfo001.obj
 0002:000009e8       ??_C@_0BL@LDIMKLPH@JVMTI_ERROR_INVALID_THREAD@ 00000001800059e8     libtimerinfo001.obj
 0002:00000a08       ??_C@_0CB@PJFPAIKJ@JVMTI_ERROR_INVALID_THREAD_GROU@ 0000000180005a08     libtimerinfo001.obj
 0002:00000a30       ??_C@_0BN@LLMKHMNF@JVMTI_ERROR_INVALID_PRIORITY@ 0000000180005a30     libtimerinfo001.obj
 0002:00000a50       ??_C@_0CB@MBOFKAGB@JVMTI_ERROR_THREAD_NOT_SUSPENDE@ 0000000180005a50     libtimerinfo001.obj
 0002:00000a78       ??_C@_0BN@FABOLPBI@JVMTI_ERROR_THREAD_SUSPENDED@ 0000000180005a78     libtimerinfo001.obj
 0002:00000a98       ??_C@_0BN@FDGNOBJM@JVMTI_ERROR_THREAD_NOT_ALIVE@ 0000000180005a98     libtimerinfo001.obj
 0002:00000ab8       ??_C@_0BL@GOBIFKNJ@JVMTI_ERROR_INVALID_OBJECT@ 0000000180005ab8     libtimerinfo001.obj
 0002:00000ad8       ??_C@_0BK@FCMAJPPC@JVMTI_ERROR_INVALID_CLASS@ 0000000180005ad8     libtimerinfo001.obj
 0002:00000af8       ??_C@_0BP@IKLLBKEB@JVMTI_ERROR_CLASS_NOT_PREPARED@ 0000000180005af8     libtimerinfo001.obj
 0002:00000b18       ??_C@_0BN@KLPPLKG@JVMTI_ERROR_INVALID_METHODID@ 0000000180005b18     libtimerinfo001.obj
 0002:00000b38       ??_C@_0BN@BCEKOKND@JVMTI_ERROR_INVALID_LOCATION@ 0000000180005b38     libtimerinfo001.obj
 0002:00000b58       ??_C@_0BM@DFDGPME@JVMTI_ERROR_INVALID_FIELDID@ 0000000180005b58     libtimerinfo001.obj
 0002:00000b78       ??_C@_0BL@NELIEPEC@JVMTI_ERROR_NO_MORE_FRAMES@ 0000000180005b78     libtimerinfo001.obj
 0002:00000b98       ??_C@_0BJ@BDBECFDM@JVMTI_ERROR_OPAQUE_FRAME@ 0000000180005b98     libtimerinfo001.obj
 0002:00000bb8       ??_C@_0BK@MIIFNLOB@JVMTI_ERROR_TYPE_MISMATCH@ 0000000180005bb8     libtimerinfo001.obj
 0002:00000bd8       ??_C@_0BJ@HPCAOILC@JVMTI_ERROR_INVALID_SLOT@ 0000000180005bd8     libtimerinfo001.obj
 0002:00000bf8       ??_C@_0BG@CHILOPNI@JVMTI_ERROR_DUPLICATE@ 0000000180005bf8     libtimerinfo001.obj
 0002:00000c10       ??_C@_0BG@DIEMLHKM@JVMTI_ERROR_NOT_FOUND@ 0000000180005c10     libtimerinfo001.obj
 0002:00000c28       ??_C@_0BM@NHMCKHOB@JVMTI_ERROR_INVALID_MONITOR@ 0000000180005c28     libtimerinfo001.obj
 0002:00000c48       ??_C@_0BO@PPEDAJGL@JVMTI_ERROR_NOT_MONITOR_OWNER@ 0000000180005c48     libtimerinfo001.obj
 0002:00000c68       ??_C@_0BG@FCAIPEID@JVMTI_ERROR_INTERRUPT@ 0000000180005c68     libtimerinfo001.obj
 0002:00000c80       ??_C@_0CB@EGDBNKOI@JVMTI_ERROR_INVALID_CLASS_FORMA@ 0000000180005c80     libtimerinfo001.obj
 0002:00000ca8       ??_C@_0CG@DGKOGIAL@JVMTI_ERROR_CIRCULAR_CLASS_DEFI@ 0000000180005ca8     libtimerinfo001.obj
 0002:00000cd0       ??_C@_0BP@ICEALPKC@JVMTI_ERROR_FAILS_VERIFICATION@ 0000000180005cd0     libtimerinfo001.obj
 0002:00000cf0       ??_C@_0DC@JDACLMIO@JVMTI_ERROR_UNSUPPORTED_REDEFIN@ 0000000180005cf0     libtimerinfo001.obj
 0002:00000d28       ??_C@_0DE@GKDKNOMJ@JVMTI_ERROR_UNSUPPORTED_REDEFIN@ 0000000180005d28     libtimerinfo001.obj
 0002:00000d60       ??_C@_0BO@LAFKIOG@JVMTI_ERROR_INVALID_TYPESTATE@ 0000000180005d60     libtimerinfo001.obj
 0002:00000d80       ??_C@_0DH@INDGCLLB@JVMTI_ERROR_UNSUPPORTED_REDEFIN@ 0000000180005d80     libtimerinfo001.obj
 0002:00000db8       ??_C@_0DE@NHEOMMGI@JVMTI_ERROR_UNSUPPORTED_REDEFIN@ 0000000180005db8     libtimerinfo001.obj
 0002:00000df0       ??_C@_0CA@EKPNJOEP@JVMTI_ERROR_UNSUPPORTED_VERSION@ 0000000180005df0     libtimerinfo001.obj
 0002:00000e10       ??_C@_0BN@OFFMAHHL@JVMTI_ERROR_NAMES_DONT_MATCH@ 0000000180005e10     libtimerinfo001.obj
 0002:00000e30       ??_C@_0DN@HHBBLAKE@JVMTI_ERROR_UNSUPPORTED_REDEFIN@ 0000000180005e30     libtimerinfo001.obj
 0002:00000e70       ??_C@_0DO@HMBGBGNA@JVMTI_ERROR_UNSUPPORTED_REDEFIN@ 0000000180005e70     libtimerinfo001.obj
 0002:00000eb0       ??_C@_0BP@PBECGKHJ@JVMTI_ERROR_UNMODIFIABLE_CLASS@ 0000000180005eb0     libtimerinfo001.obj
 0002:00000ed0       ??_C@_0BK@CANILEHF@JVMTI_ERROR_NOT_AVAILABLE@ 0000000180005ed0     libtimerinfo001.obj
 0002:00000ef0       ??_C@_0CE@INJKMEFK@JVMTI_ERROR_MUST_POSSESS_CAPABI@ 0000000180005ef0     libtimerinfo001.obj
 0002:00000f18       ??_C@_0BJ@LBFPFPDM@JVMTI_ERROR_NULL_POINTER@ 0000000180005f18     libtimerinfo001.obj
 0002:00000f38       ??_C@_0BP@CHJPNNEM@JVMTI_ERROR_ABSENT_INFORMATION@ 0000000180005f38     libtimerinfo001.obj
 0002:00000f58       ??_C@_0BP@OMFMNLC@JVMTI_ERROR_INVALID_EVENT_TYPE@ 0000000180005f58     libtimerinfo001.obj
 0002:00000f78       ??_C@_0BN@BIBNPHHO@JVMTI_ERROR_ILLEGAL_ARGUMENT@ 0000000180005f78     libtimerinfo001.obj
 0002:00000f98       ??_C@_0BK@KKNDHDCE@JVMTI_ERROR_NATIVE_METHOD@ 0000000180005f98     libtimerinfo001.obj
 0002:00000fb8       ??_C@_0BK@PMKCFHAE@JVMTI_ERROR_OUT_OF_MEMORY@ 0000000180005fb8     libtimerinfo001.obj
 0002:00000fd8       ??_C@_0BK@NNJBDMNB@JVMTI_ERROR_ACCESS_DENIED@ 0000000180005fd8     libtimerinfo001.obj
 0002:00000ff8       ??_C@_0BI@GHECLMNC@JVMTI_ERROR_WRONG_PHASE@ 0000000180005ff8     libtimerinfo001.obj
 0002:00001010       ??_C@_0BF@OLIHJOII@JVMTI_ERROR_INTERNAL@ 0000000180006010     libtimerinfo001.obj
 0002:00001028       ??_C@_0BO@EOHGKJHI@JVMTI_ERROR_UNATTACHED_THREAD@ 0000000180006028     libtimerinfo001.obj
 0002:00001048       ??_C@_0CA@LKHFDACL@JVMTI_ERROR_INVALID_ENVIRONMENT@ 0000000180006048     libtimerinfo001.obj
 0002:00001068       ??_C@_0BA@MMFHLOKK@?$DMunknown?5error?$DO@ 0000000180006068     libtimerinfo001.obj
 0002:00001078       ??_C@_0CF@CBHOKDB@throwable?5?$DN?5jni?9?$DOExceptionOccur@ 0000000180006078     libtimerinfo001.obj
 0002:000010a0       ??_C@_03OFAPEBGM@?$CFs?6@  00000001800060a0     libtimerinfo001.obj
 0002:000010a8       ??_C@_0DM@LPIGEGNJ@s?2test?2hotspot?2jtreg?2vmTestbase@ 00000001800060a8     libtimerinfo001.obj
 0002:000010e8       ??_C@_0CC@NFCNPEPK@Exception?5in?5JNI?5call?5?$CIcleared?$CJ@ 00000001800060e8     libtimerinfo001.obj
 0002:00001110       ??_C@_0BJ@IBAKFIKF@jni?9?$DOExceptionDescribe?$CI?$CJ@ 0000000180006110     libtimerinfo001.obj
 0002:00001130       ??_C@_0BG@GGKALKMH@jni?9?$DOExceptionClear?$CI?$CJ@ 0000000180006130     libtimerinfo001.obj
 0002:00001148       ??_C@_0CF@JMGFGJLJ@?$CD?5?5?5verified?5JNI?5assertion?5is?5F@ 0000000180006148     libtimerinfo001.obj
 0002:00001170       ??_C@_07KBAMPNJK@verbose@  0000000180006170     libtimerinfo001.obj
 0002:00001178       ??_C@_0DN@PKJBOLAP@nsk_jvmti_parseOptions?$CI?$CJ?3?5unexp@ 0000000180006178     libtimerinfo001.obj
 0002:000011b8       ??_C@_05IMBNNINJ@trace@    00000001800061b8     libtimerinfo001.obj
 0002:000011c0       ??_C@_0DD@BJKGNDMB@nsk_jvmti_parseOptions?$CI?$CJ?3?5no?5va@ 00000001800061c0     libtimerinfo001.obj
 0002:000011f4       ??_C@_04CGFJFPFD@none@     00000001800061f4     libtimerinfo001.obj
 0002:000011fc       ??_C@_06BMELKFMA@before@   00000001800061fc     libtimerinfo001.obj
 0002:00001204       ??_C@_05CMKPCFDK@after@    0000000180006204     libtimerinfo001.obj
 0002:0000120c       ??_C@_03NFKEKGGK@all@      000000018000620c     libtimerinfo001.obj
 0002:00001210       ??_C@_0DM@NDNJGJKE@nsk_jvmti_parseOptions?$CI?$CJ?3?5uexpe@ 0000000180006210     libtimerinfo001.obj
 0002:00001250       ??_C@_08NBBJKJO@waittime@  0000000180006250     libtimerinfo001.obj
 0002:00001260       ??_C@_0DO@CMHGAOHC@nsk_jvmti_parseOptions?$CI?$CJ?3?5not?5i@ 0000000180006260     libtimerinfo001.obj
 0002:000012a0       ??_C@_0DL@LNMPBDLN@nsk_jvmti_parseOptions?$CI?$CJ?3?5negat@ 00000001800062a0     libtimerinfo001.obj
 0002:000012e0       ??_C@_0DA@GMFJNOJH@nsk_jvmti_parseOptions?$CI?$CJ?3?5unkno@ 00000001800062e0     libtimerinfo001.obj
 0002:00001310       ??_C@_0CO@CCIAMEAN@nsk_jvmti_parseOptions?$CI?$CJ?3?5found@ 0000000180006310     libtimerinfo001.obj
 0002:00001340       ??_C@_0CJ@OEGPCGDL@nsk_jvmti_parseOptions?$CI?$CJ?3?5out?5o@ 0000000180006340     libtimerinfo001.obj
 0002:00001370       ??_C@_0DI@NMBHPGGF@nsk_jvmti_parseOptions?$CI?$CJ?3?5too?5m@ 0000000180006370     libtimerinfo001.obj
 0002:000013a8       ??_C@_03POGCGECB@?5?0?$HO@ 00000001800063a8     libtimerinfo001.obj
 0002:000013b0       ??_C@_0CB@MLNJNCLJ@?5?5jvmti?5error?3?5code?$DN?$CFd?0?5name?$DN?$CFs@ 00000001800063b0     libtimerinfo001.obj
 0002:000013d8       ??_C@_0CD@OHBGDKMK@?$CD?5?5?5jvmti?5error?3?5code?$DN?$CFd?0?5name?$DN@ 00000001800063d8     libtimerinfo001.obj
 0002:00001400       ??_C@_0CG@JNNCGPHB@?$CD?5?5?5error?5expected?3?5code?$DN?$CFd?0?5na@ 0000000180006400     libtimerinfo001.obj
 0002:00001430       ??_C@_0EB@IMGKPCGE@?$CIstr_obj?5?$DN?5jni?9?$DONewStringUTF?$CIco@ 0000000180006430     libtimerinfo001.obj
 0002:00001480       ??_C@_0EA@HFOGGBCC@s?2test?2hotspot?2jtreg?2vmTestbase@ 0000000180006480     libtimerinfo001.obj
 0002:000014c0       ??_C@_05KKCIMGE@error@     00000001800064c0     libtimerinfo001.obj
 0002:000014c8       ??_C@_0BD@HGNAOMCP@agent_data_monitor@ 00000001800064c8     libtimerinfo001.obj
 0002:000014e0       ??_C@_0EB@OGCLGKLN@javaVM?9?$DOGetEnv?$CI?$CIvoid?5?$CK?$CK?$CJ?$CGjvmti_@ 00000001800064e0     libtimerinfo001.obj
 0002:00001530       ??_C@_0EA@PNBCDMOA@s?2test?2hotspot?2jtreg?2vmTestbase@ 0000000180006530     libtimerinfo001.obj
 0002:00001570       ??_C@_0CI@DDPIFBGM@init_agent_data?$CIjvmti_env?0?5?$CGage@ 0000000180006570     libtimerinfo001.obj
 0002:00001598       ??_C@_0DI@ILAHDLMP@?$CI?$CKagentThreadProc?$CJ?$CIjvmti_env?0?5a@ 0000000180006598     libtimerinfo001.obj
 0002:000015d0       ??_C@_0BD@KDBALNLB@JVMTI?5agent?5thread@ 00000001800065d0     libtimerinfo001.obj
 0002:000015e8       ??_C@_0BB@NOKBFPFO@java?1lang?1Thread@ 00000001800065e8     libtimerinfo001.obj
 0002:000015fc       ??_C@_06FALKBLGB@?$DMinit?$DO@ 00000001800065fc     libtimerinfo001.obj
 0002:00001608       ??_C@_0BG@IKDDPPGD@?$CILjava?1lang?1String?$DL?$CJV@ 0000000180006608     libtimerinfo001.obj
 0002:00001620       ??_C@_0EB@IFJBFEKC@?$CIthreadClass?5?$DN?5jni_env?9?$DOFindCla@ 0000000180006620     libtimerinfo001.obj
 0002:00001670       ??_C@_0GF@FGFIBKKL@?$CIthreadCtor?5?$DN?5jni_env?9?$DOGetMetho@ 0000000180006670     libtimerinfo001.obj
 0002:000016d8       ??_C@_0DN@NCPDJLOG@?$CIthreadName?5?$DN?5jni_env?9?$DONewStrin@ 00000001800066d8     libtimerinfo001.obj
 0002:00001720       ??_C@_0FE@PFKODBGC@?$CIthreadObject?5?$DN?5jni_env?9?$DONewObj@ 0000000180006720     libtimerinfo001.obj
 0002:00001780       ??_C@_0ED@HOBAHHJI@?$CIthreadGlobalRef?5?$DN?5jni_env?9?$DONew@ 0000000180006780     libtimerinfo001.obj
 0002:000017d0       ??_C@_0FN@HNJJAHFC@jvmti_env?9?$DORunAgentThread?$CIagent@ 00000001800067d0     libtimerinfo001.obj
 0002:00001830       ??_C@_0EA@MOJDNKDF@Debuggee?5status?5sync?5aborted?5be@ 0000000180006830     libtimerinfo001.obj
 0002:00001870       ??_C@_0CO@PGPGMHBJ@No?5status?5sync?5occured?5for?5time@ 0000000180006870     libtimerinfo001.obj
 0002:000018a0       ??_C@_0CL@DOEBDPKJ@Debuggee?5was?5not?5suspended?5on?5s@ 00000001800068a0     libtimerinfo001.obj
 0002:000018d0       ??_C@_0EA@EEOEJAEN@status?5?$DN?5syncDebuggeeStatus?$CIjni@ 00000001800068d0     libtimerinfo001.obj
 0002:00001910       ??_C@_0BL@JBCFNBMB@nsk_jvmti_resetAgentData?$CI?$CJ@ 0000000180006910     libtimerinfo001.obj
 0002:00001930       ??_C@_0DN@NNGECJON@jvmti_env?9?$DOSetEventNotification@ 0000000180006930     libtimerinfo001.obj
 0002:00001970       ??_C@_0EL@LPBEELIP@s?2test?2hotspot?2jtreg?2vmTestbase@ 0000000180006970     libtimerinfo001.obj
 0002:000019c0       ??_C@_0CK@JDAMFDMJ@jvmti?9?$DOSetTag?$CIo?0?5tag?$CJ?5?$DN?$DN?5JVMTI_@ 00000001800069c0     libtimerinfo001.obj
 0002:000019f0       ??_C@_0CC@DAMNHKNI@Can?8t?5set?5tag?5?$CFli?5for?5object?5?$CFl@ 00000001800069f0     libtimerinfo001.obj
 0002:00001a18       ??_C@_0DL@HAJPNKEF@jvmti?9?$DOGetObjectHashCode?$CIo?0?5?$CGha@ 0000000180006a18     libtimerinfo001.obj
 0002:00001a58       ??_C@_0BL@JFPIEOBF@Can?8t?5get?5hash?5object?5?$CFlx?6@ 0000000180006a58     libtimerinfo001.obj
 0002:00001a78       ??_C@_0BG@DICPHBKN@setTag?3?5?$CF08x?5?$DM?9?5?$CF?53li@ 0000000180006a78     libtimerinfo001.obj
 0002:00001a90       ??_C@_0DH@FCEEBDMJ@?$CIs?5?$DN?5jni?9?$DOGetStringUTFChars?$CIsIn@ 0000000180006a90     libtimerinfo001.obj
 0002:00001ac8       ??_C@_0BJ@OKKGHDCN@Can?8t?5get?5string?5at?5?$CF?$CDp?6@ 0000000180006ac8     libtimerinfo001.obj
 0002:00001ae8       ??_C@_0BP@EKFLGGFJ@Can?8t?5get?5string?5at?5?$CF?$CDp?3?5null?6@ 0000000180006ae8     libtimerinfo001.obj
 0002:00001b08       ??_C@_06ICODBHCL@?5?1?1?5?$CFs@ 0000000180006b08     libtimerinfo001.obj
 0002:00001b10       ??_C@_0DB@KGFPLEGO@?$CIr?5?$DN?5jvmti?9?$DOGetTag?$CIo?0?5?$CGtag?$CJ?$CJ?5?$DN?$DN@ 0000000180006b10     libtimerinfo001.obj
 0002:00001b48       ??_C@_0CO@PDAGBCGJ@Can?8t?5GetTag?5for?5object?5?$CFlx?4?5Re@ 0000000180006b48     libtimerinfo001.obj
 0002:00001b78       ??_C@_0CH@HPEODOHC@TEST_BUG?3?5Max?4?5number?5of?5refs?5r@ 0000000180006b78     libtimerinfo001.obj
 0002:00001ba0       ??_C@_0DI@PHFCABIM@?$CIr?5?$DN?5jvmti?9?$DOGetTag?$CIfrom?0?5?$CGtagFr@ 0000000180006ba0     libtimerinfo001.obj
 0002:00001bd8       ??_C@_0DI@MDEGFNKD@TEST_BUG?3?5Can?8t?5GetTag?5for?5obje@ 0000000180006bd8     libtimerinfo001.obj
 0002:00001c10       ??_C@_0DE@MLELJAHM@?$CIr?5?$DN?5jvmti?9?$DOGetTag?$CIto?0?5?$CGtagTo?$CJ?$CJ@ 0000000180006c10     libtimerinfo001.obj
 0002:00001c48       ??_C@_0CG@NEHINGLM@GetTimerInfo?$CI?$CJ?5for?5current?5JVMT@ 0000000180006c48     libtimerinfo001.obj
 0002:00001c70       ??_C@_0FF@ENNOMDMG@s?2test?2hotspot?2jtreg?2vmTestbase@ 0000000180006c70     libtimerinfo001.obj
 0002:00001cc8       ??_C@_0BK@MEFDANLG@jvmti?9?$DOGetTimerInfo?$CIinfo?$CJ@ 0000000180006cc8     libtimerinfo001.obj
 0002:00001ce8       ??_C@_0BB@HDMEGNLK@Got?5timer?5info?3?6@ 0000000180006ce8     libtimerinfo001.obj
 0002:00001d00       ??_C@_0BL@HIODFFAA@?5?5?5?5max_value?3?5?5?5?5?5?5?5?5?5?$CFs?6@ 0000000180006d00     libtimerinfo001.obj
 0002:00001d20       ??_C@_0BL@KCGDNOOA@?5?5?5?5may_skip_forward?3?5?5?$CFd?6@ 0000000180006d20     libtimerinfo001.obj
 0002:00001d40       ??_C@_0BL@KGPGKOHE@?5?5?5?5may_skip_backward?3?5?$CFd?6@ 0000000180006d40     libtimerinfo001.obj
 0002:00001d60       ??_C@_0CB@CBFDDKLG@Compare?5with?5initial?5timer?5info@ 0000000180006d60     libtimerinfo001.obj
 0002:00001d88       ??_C@_09JLDFFDBG@max_value@ 0000000180006d88     libtimerinfo001.obj
 0002:00001da0       ??_C@_0GF@NINCAIGP@In?5?$CFs?5GetTimerInfo?$CI?$CJ?5returned?5d@ 0000000180006da0     libtimerinfo001.obj
 0002:00001e08       ??_C@_0BB@FMAKKIPA@may_skip_forward@ 0000000180006e08     libtimerinfo001.obj
 0002:00001e20       ??_C@_0GF@ODLICJCO@In?5?$CFs?5GetTimerInfo?$CI?$CJ?5returned?5d@ 0000000180006e20     libtimerinfo001.obj
 0002:00001e88       ??_C@_0BC@PEAMAFCC@may_skip_backward@ 0000000180006e88     libtimerinfo001.obj
 0002:00001ea0       ??_C@_0CC@HCPFMLEK@Wait?5for?5debugee?5to?5become?5read@ 0000000180006ea0     libtimerinfo001.obj
 0002:00001ec8       ??_C@_0DD@OJKMPBLI@?$DO?$DO?$DO?5Testcase?5?$CD3?3?5Check?5timer?5in@ 0000000180006ec8     libtimerinfo001.obj
 0002:00001f00       ??_C@_0N@POFOADDC@agent?5thread@ 0000000180006f00     libtimerinfo001.obj
 0002:00001f10       ??_C@_0BH@HPEOJMHL@Let?5debugee?5to?5finish?6@ 0000000180006f10     libtimerinfo001.obj
 0002:00001f28       ??_C@_0DH@KJMEEBGF@?$DO?$DO?$DO?5Testcase?5?$CD2?3?5Check?5timer?5in@ 0000000180006f28     libtimerinfo001.obj
 0002:00001f60       ??_C@_0BB@ECBNOENI@VM_INIT?5callback@ 0000000180006f60     libtimerinfo001.obj
 0002:00001f78       ??_C@_0DI@OHIKNEHC@?$DO?$DO?$DO?5Testcase?5?$CD4?3?5Check?5timer?5in@ 0000000180006f78     libtimerinfo001.obj
 0002:00001fb0       ??_C@_0BC@BEKPBLPI@VM_DEATH?5callback@ 0000000180006fb0     libtimerinfo001.obj
 0002:00001fc8       ??_C@_0BL@OGOOPPCN@Disable?5events?3?5?$CFd?5events?6@ 0000000180006fc8     libtimerinfo001.obj
 0002:00001fe8       ??_C@_0BA@DDKAOGOI@?5?5?4?4?4?5disabled?6@ 0000000180006fe8     libtimerinfo001.obj
 0002:00001ff8       ??_C@_0CA@LDMJDFDO@Exit?5with?5FAIL?5exit?5status?3?5?$CFd?6@ 0000000180006ff8     libtimerinfo001.obj
 0002:00002018       ??_C@_0BC@PCOLJFHD@exit?$CISTATUS_FAIL?$CJ@ 0000000180007018     libtimerinfo001.obj
 0002:00002030       ??_C@_0CA@MNKGCBCG@nsk_jvmti_parseOptions?$CIoptions?$CJ@ 0000000180007030     libtimerinfo001.obj
 0002:00002050       ??_C@_0DN@MIAMNFPH@?$CIjvmti?5?$DN?5nsk_jvmti_createJVMTIE@ 0000000180007050     libtimerinfo001.obj
 0002:00002090       ??_C@_0EC@ODFGFOAJ@jvmti?9?$DOSetEventCallbacks?$CI?$CGevent@ 0000000180007090     libtimerinfo001.obj
 0002:000020d8       ??_C@_0CL@PIACJIPK@nsk_jvmti_setAgentProc?$CIagentPro@ 00000001800070d8     libtimerinfo001.obj
 0002:00002108       ??_C@_0DN@BBNFPMPE@?$DO?$DO?$DO?5Testcase?5?$CD1?3?5Check?5initial?5@ 0000000180007108     libtimerinfo001.obj
 0002:00002148       ??_C@_0P@LKCKDJEM@Agent_OnLoad?$CI?$CJ@ 0000000180007148     libtimerinfo001.obj
 0002:00002158       ??_C@_0BK@EKNILGAD@Enable?5events?3?5?$CFd?5events?6@ 0000000180007158     libtimerinfo001.obj
 0002:00002178       ??_C@_0P@BAMBNLJF@?5?5?4?4?4?5enabled?6@ 0000000180007178     libtimerinfo001.obj
 0002:000021a0       ??_C@_1EC@JIJBPKFM@?$AAa?$AAp?$AAi?$AA?9?$AAm?$AAs?$AA?9?$AAw?$AAi?$AAn?$AA?9?$AAc?$AAo?$AAr?$AAe@ 00000001800071a0     MSVCRT:thread_safe_statics.obj
 0002:000021e8       ??_C@_1BK@MGMFAEKH@?$AAk?$AAe?$AAr?$AAn?$AAe?$AAl?$AA3?$AA2?$AA?4?$AAd?$AAl?$AAl@ 00000001800071e8     MSVCRT:thread_safe_statics.obj
 0002:00002208       ??_C@_0BJ@JEBJOJFJ@SleepConditionVariableCS@ 0000000180007208     MSVCRT:thread_safe_statics.obj
 0002:00002228       ??_C@_0BJ@PGPPEPCC@WakeAllConditionVariable@ 0000000180007228     MSVCRT:thread_safe_statics.obj
 0002:00002248       _pDefaultRawDllMain        0000000180007248     MSVCRT:dll_dllmain.obj
 0002:00002248       _pRawDllMain               0000000180007248     MSVCRT:dll_dllmain.obj
 0002:00002250       __xmm@ffffffffffffffffffffffffffffffff 0000000180007250     MSVCRT:utility.obj
 0002:00002260       _load_config_used          0000000180007260     MSVCRT:loadcfg.obj
 0002:00002480       _tls_used                  0000000180007480     MSVCRT:tlssup.obj
 0002:000024a8       __volatile_metadata        00000001800074a8     <linker-defined>
 0002:000028a8       __rtc_iaa                  00000001800078a8     MSVCRT:initsect.obj
 0002:000028b0       __rtc_izz                  00000001800078b0     MSVCRT:initsect.obj
 0002:000028b8       __rtc_taa                  00000001800078b8     MSVCRT:initsect.obj
 0002:000028c0       __rtc_tzz                  00000001800078c0     MSVCRT:initsect.obj
 0002:000028c8       _tls_start                 00000001800078c8     MSVCRT:tlssup.obj
 0002:000028cc       _Init_thread_epoch         00000001800078cc     MSVCRT:thread_safe_statics.obj
 0002:000028d0       _tls_end                   00000001800078d0     MSVCRT:tlssup.obj
 0002:00003008       __IMPORT_DESCRIPTOR_KERNEL32 0000000180008008     kernel32:KERNEL32.dll
 0002:0000301c       __IMPORT_DESCRIPTOR_VCRUNTIME140 000000018000801c     vcruntime:VCRUNTIME140.dll
 0002:00003030       __IMPORT_DESCRIPTOR_api-ms-win-crt-heap-l1-1-0 0000000180008030     ucrt:api-ms-win-crt-heap-l1-1-0.dll
 0002:00003044       __IMPORT_DESCRIPTOR_api-ms-win-crt-runtime-l1-1-0 0000000180008044     ucrt:api-ms-win-crt-runtime-l1-1-0.dll
 0002:00003058       __IMPORT_DESCRIPTOR_api-ms-win-crt-convert-l1-1-0 0000000180008058     ucrt:api-ms-win-crt-convert-l1-1-0.dll
 0002:0000306c       __IMPORT_DESCRIPTOR_api-ms-win-crt-stdio-l1-1-0 000000018000806c     ucrt:api-ms-win-crt-stdio-l1-1-0.dll
 0002:00003080       __IMPORT_DESCRIPTOR_api-ms-win-crt-string-l1-1-0 0000000180008080     ucrt:api-ms-win-crt-string-l1-1-0.dll
 0002:00003094       __NULL_IMPORT_DESCRIPTOR   0000000180008094     kernel32:KERNEL32.dll
 0003:00000038       _Init_global_epoch         0000000180009038     MSVCRT:thread_safe_statics.obj
 0003:00000040       __security_cookie          0000000180009040     MSVCRT:gs_cookie.obj
 0003:00000048       __security_cookie_complement 0000000180009048     MSVCRT:gs_cookie.obj
 0003:00000050       __scrt_native_dllmain_reason 0000000180009050     MSVCRT:utility.obj
 0003:00000058       __isa_available            0000000180009058     MSVCRT:cpu_disp.obj
 0003:0000005c       __isa_enabled              000000018000905c     MSVCRT:cpu_disp.obj
 0003:00000060       __memset_fast_string_threshold 0000000180009060     MSVCRT:cpu_disp.obj
 0003:00000068       __memset_nt_threshold      0000000180009068     MSVCRT:cpu_disp.obj
 0003:00000070       __scrt_ucrt_dll_is_in_use  0000000180009070     MSVCRT:ucrt_stubs.obj
 0003:00000080       g_wrongHeapCallbacks       0000000180009080     libtimerinfo001.obj
 0003:00000100       g_szTagInfo                0000000180009100     libtimerinfo001.obj
 0003:00002040       g_tagFlags                 000000018000b040     libtimerinfo001.obj
 0003:00002428       g_refsToVerifyCnt          000000018000b428     libtimerinfo001.obj
 0003:0000242c       g_fakeUserData             000000018000b42c     libtimerinfo001.obj
 0003:00002430       g_tagVisitCount            000000018000b430     libtimerinfo001.obj
 0003:000033d0       g_refsToVerify             000000018000c3d0     libtimerinfo001.obj
 0003:0001aad0       g_userDataError            0000000180023ad0     libtimerinfo001.obj
 0003:0001ac90       ?_OptionsStorage@?1??__local_stdio_printf_options@@9@4_KA 0000000180023c90     libtimerinfo001.obj
 0003:0001b258       _tls_index                 0000000180024258     MSVCRT:tlssup.obj
 0003:0001b260       __scrt_current_native_startup_state 0000000180024260     MSVCRT:utility.obj
 0003:0001b268       __scrt_native_startup_lock 0000000180024268     MSVCRT:utility.obj
 0003:0001b2a8       __scrt_debugger_hook_flag  00000001800242a8     MSVCRT:utility_desktop.obj
 0003:0001b2b0       ?__type_info_root_node@@3U__type_info_node@@A 00000001800242b0     MSVCRT:tncleanup.obj
 0003:0001b2c0       ?_OptionsStorage@?1??__local_stdio_scanf_options@@9@4_KA 00000001800242c0     MSVCRT:default_local_stdio_options.obj
 0003:0001b2c8       __favor                    00000001800242c8     MSVCRT:cpu_disp.obj
 0003:0001b2d0       __dyn_tls_init_callback    00000001800242d0     <common>

 entry point at        0001:00002ef0

 Static symbols

 0000:fffd9000       .debug$S                   0000000180000000     timerinfo001.exp
 0000:fffd9000       .debug$S                   0000000180000000     vcruntime:VCRUNTIME140.dll
 0000:fffd9000       .debug$S                   0000000180000000     vcruntime:VCRUNTIME140.dll
 0000:fffd9000       .debug$S                   0000000180000000     vcruntime:VCRUNTIME140.dll
 0000:fffd9000       .debug$S                   0000000180000000     vcruntime:VCRUNTIME140.dll
 0000:fffd9000       .debug$S                   0000000180000000     vcruntime:VCRUNTIME140.dll
 0000:fffd9000       .debug$S                   0000000180000000     vcruntime:VCRUNTIME140.dll
 0000:fffd9000       .debug$S                   0000000180000000     vcruntime:VCRUNTIME140.dll
 0000:fffd9000       .debug$S                   0000000180000000     ucrt:api-ms-win-crt-convert-l1-1-0.dll
 0000:fffd9000       .debug$S                   0000000180000000     ucrt:api-ms-win-crt-heap-l1-1-0.dll
 0000:fffd9000       .debug$S                   0000000180000000     ucrt:api-ms-win-crt-heap-l1-1-0.dll
 0000:fffd9000       .debug$S                   0000000180000000     ucrt:api-ms-win-crt-heap-l1-1-0.dll
 0000:fffd9000       .debug$S                   0000000180000000     ucrt:api-ms-win-crt-heap-l1-1-0.dll
 0000:fffd9000       .debug$S                   0000000180000000     ucrt:api-ms-win-crt-runtime-l1-1-0.dll
 0000:fffd9000       .debug$S                   0000000180000000     ucrt:api-ms-win-crt-runtime-l1-1-0.dll
 0000:fffd9000       .debug$S                   0000000180000000     ucrt:api-ms-win-crt-runtime-l1-1-0.dll
 0000:fffd9000       .debug$S                   0000000180000000     ucrt:api-ms-win-crt-runtime-l1-1-0.dll
 0000:fffd9000       .debug$S                   0000000180000000     ucrt:api-ms-win-crt-runtime-l1-1-0.dll
 0000:fffd9000       .debug$S                   0000000180000000     ucrt:api-ms-win-crt-runtime-l1-1-0.dll
 0000:fffd9000       .debug$S                   0000000180000000     ucrt:api-ms-win-crt-runtime-l1-1-0.dll
 0000:fffd9000       .debug$S                   0000000180000000     ucrt:api-ms-win-crt-runtime-l1-1-0.dll
 0000:fffd9000       .debug$S                   0000000180000000     ucrt:api-ms-win-crt-runtime-l1-1-0.dll
 0000:fffd9000       .debug$S                   0000000180000000     ucrt:api-ms-win-crt-runtime-l1-1-0.dll
 0000:fffd9000       .debug$S                   0000000180000000     ucrt:api-ms-win-crt-runtime-l1-1-0.dll
 0000:fffd9000       .debug$S                   0000000180000000     ucrt:api-ms-win-crt-runtime-l1-1-0.dll
 0000:fffd9000       .debug$S                   0000000180000000     ucrt:api-ms-win-crt-runtime-l1-1-0.dll
 0000:fffd9000       .debug$S                   0000000180000000     ucrt:api-ms-win-crt-runtime-l1-1-0.dll
 0000:fffd9000       .debug$S                   0000000180000000     ucrt:api-ms-win-crt-runtime-l1-1-0.dll
 0000:fffd9000       .debug$S                   0000000180000000     ucrt:api-ms-win-crt-runtime-l1-1-0.dll
 0000:fffd9000       .debug$S                   0000000180000000     ucrt:api-ms-win-crt-stdio-l1-1-0.dll
 0000:fffd9000       .debug$S                   0000000180000000     ucrt:api-ms-win-crt-stdio-l1-1-0.dll
 0000:fffd9000       .debug$S                   0000000180000000     ucrt:api-ms-win-crt-stdio-l1-1-0.dll
 0000:fffd9000       .debug$S                   0000000180000000     ucrt:api-ms-win-crt-stdio-l1-1-0.dll
 0000:fffd9000       .debug$S                   0000000180000000     ucrt:api-ms-win-crt-stdio-l1-1-0.dll
 0000:fffd9000       .debug$S                   0000000180000000     ucrt:api-ms-win-crt-stdio-l1-1-0.dll
 0000:fffd9000       .debug$S                   0000000180000000     ucrt:api-ms-win-crt-stdio-l1-1-0.dll
 0000:fffd9000       .debug$S                   0000000180000000     ucrt:api-ms-win-crt-stdio-l1-1-0.dll
 0000:fffd9000       .debug$S                   0000000180000000     ucrt:api-ms-win-crt-stdio-l1-1-0.dll
 0000:fffd9000       .debug$S                   0000000180000000     ucrt:api-ms-win-crt-stdio-l1-1-0.dll
 0000:fffd9000       .debug$S                   0000000180000000     ucrt:api-ms-win-crt-string-l1-1-0.dll
 0000:fffd9000       .debug$S                   0000000180000000     ucrt:api-ms-win-crt-string-l1-1-0.dll
 0000:fffd9000       .debug$S                   0000000180000000     ucrt:api-ms-win-crt-string-l1-1-0.dll
 0000:fffd9000       .debug$S                   0000000180000000     ucrt:api-ms-win-crt-string-l1-1-0.dll
 0000:fffd9000       .debug$S                   0000000180000000     ucrt:api-ms-win-crt-string-l1-1-0.dll
 0000:fffd9000       .debug$S                   0000000180000000     ucrt:api-ms-win-crt-string-l1-1-0.dll
 0000:fffd9000       .debug$S                   0000000180000000     ucrt:api-ms-win-crt-string-l1-1-0.dll
 0000:fffd9000       .debug$S                   0000000180000000     ucrt:api-ms-win-crt-string-l1-1-0.dll
 0000:fffd9000       .debug$S                   0000000180000000     kernel32:KERNEL32.dll
 0000:fffd9000       .debug$S                   0000000180000000     kernel32:KERNEL32.dll
 0000:fffd9000       .debug$S                   0000000180000000     kernel32:KERNEL32.dll
 0000:fffd9000       .debug$S                   0000000180000000     kernel32:KERNEL32.dll
 0000:fffd9000       .debug$S                   0000000180000000     kernel32:KERNEL32.dll
 0000:fffd9000       .debug$S                   0000000180000000     kernel32:KERNEL32.dll
 0000:fffd9000       .debug$S                   0000000180000000     kernel32:KERNEL32.dll
 0000:fffd9000       .debug$S                   0000000180000000     kernel32:KERNEL32.dll
 0000:fffd9000       .debug$S                   0000000180000000     kernel32:KERNEL32.dll
 0000:fffd9000       .debug$S                   0000000180000000     kernel32:KERNEL32.dll
 0000:fffd9000       .debug$S                   0000000180000000     kernel32:KERNEL32.dll
 0000:fffd9000       .debug$S                   0000000180000000     kernel32:KERNEL32.dll
 0000:fffd9000       .debug$S                   0000000180000000     kernel32:KERNEL32.dll
 0000:fffd9000       .debug$S                   0000000180000000     kernel32:KERNEL32.dll
 0000:fffd9000       .debug$S                   0000000180000000     kernel32:KERNEL32.dll
 0000:fffd9000       .debug$S                   0000000180000000     kernel32:KERNEL32.dll
 0000:fffd9000       .debug$S                   0000000180000000     kernel32:KERNEL32.dll
 0000:fffd9000       .debug$S                   0000000180000000     kernel32:KERNEL32.dll
 0000:fffd9000       .debug$S                   0000000180000000     kernel32:KERNEL32.dll
 0000:fffd9000       .debug$S                   0000000180000000     kernel32:KERNEL32.dll
 0000:fffd9000       .debug$S                   0000000180000000     kernel32:KERNEL32.dll
 0000:fffd9000       .debug$S                   0000000180000000     kernel32:KERNEL32.dll
 0000:fffd9000       .debug$S                   0000000180000000     kernel32:KERNEL32.dll
 0000:fffd9000       .debug$S                   0000000180000000     kernel32:KERNEL32.dll
 0000:fffd9000       .debug$S                   0000000180000000     kernel32:KERNEL32.dll
 0000:fffd9000       .debug$S                   0000000180000000     kernel32:KERNEL32.dll
 0000:fffd9000       .debug$S                   0000000180000000     kernel32:KERNEL32.dll
 0000:fffd9000       .debug$S                   0000000180000000     kernel32:KERNEL32.dll
 0001:00000f4c       addRefToVerify             0000000180001f4c f   libtimerinfo001.obj
 0001:00000fc0       agentProc                  0000000180001fc0 f   libtimerinfo001.obj
 0001:00001074       agentThreadWrapper         0000000180002074 f   libtimerinfo001.obj
 0001:00001330       checkTimerInfo             0000000180002330 f   libtimerinfo001.obj
 0001:0000155c       check_option               000000018000255c f   libtimerinfo001.obj
 0001:000017a4       file_basename              00000001800027a4 f   libtimerinfo001.obj
 0001:000023fc       startAgentThreadWrapper    00000001800033fc f   libtimerinfo001.obj
 0001:00002728       syncDebuggeeStatus         0000000180003728 f   libtimerinfo001.obj
 0001:000029b0       capture_previous_context   00000001800039b0 f   MSVCRT:gs_report.obj
 0001:00002a24       ?__scrt_initialize_thread_safe_statics@@YAHXZ 0000000180003a24 f   MSVCRT:thread_safe_statics.obj
 0001:00002af4       ?__scrt_uninitialize_thread_safe_statics@@YAXXZ 0000000180003af4 f   MSVCRT:thread_safe_statics.obj
 0001:00002ba0       $$000000                   0000000180003ba0     MSVCRT:amdsecgs.obj
 0001:00002bd0       ?dllmain_crt_dispatch@@YAHQEAUHINSTANCE__@@KQEAX@Z 0000000180003bd0 f   MSVCRT:dll_dllmain.obj
 0001:00002c20       ?dllmain_crt_process_attach@@YAHQEAUHINSTANCE__@@QEAX@Z 0000000180003c20 f   MSVCRT:dll_dllmain.obj
 0001:00002d38       ?dllmain_crt_process_detach@@YAH_N@Z 0000000180003d38 f   MSVCRT:dll_dllmain.obj
 0001:00002dbc       ?dllmain_dispatch@@YAHQEAUHINSTANCE__@@KQEAX@Z 0000000180003dbc f   MSVCRT:dll_dllmain.obj
 0001:000037d0       $$000000                   00000001800047d0     MSVCRT:guard_dispatch.obj
 0001:000037f0       $$000000                   00000001800047f0     MSVCRT:guard_xfg_dispatch.obj
 0001:00003806       ?fin$0@?0??dllmain_crt_process_attach@@YAHQEAUHINSTANCE__@@QEAX@Z@4HA 0000000180004806 f   MSVCRT:dll_dllmain.obj
 0001:0000381d       ?fin$0@?0??dllmain_crt_process_detach@@YAH_N@Z@4HA 000000018000481d f   MSVCRT:dll_dllmain.obj
 0001:00003836       ?fin$1@?0??dllmain_crt_process_detach@@YAH_N@Z@4HA 0000000180004836 f   MSVCRT:dll_dllmain.obj
 0001:0000384a       ?filt$0@?0??dllmain_dispatch@@YAHQEAUHINSTANCE__@@KQEAX@Z@4HA 000000018000484a f   MSVCRT:dll_dllmain.obj
 0001:00003880       __scrt_is_nonwritable_in_current_image$filt$0 0000000180004880 f   MSVCRT:utility.obj
 0002:00000218       ?__scrt_initialize_tss_var@@3P6AHXZEA 0000000180005218     MSVCRT:thread_safe_statics.obj
 0002:00000340       ?opcLengths@@3QBEB         0000000180005340     libtimerinfo001.obj
 0002:00002188       GS_ExceptionPointers       0000000180007188     MSVCRT:gs_report.obj
 0002:000028d8       $unwind$fprintf            00000001800078d8     libtimerinfo001.obj
 0002:000028e4       $unwind$printf             00000001800078e4     libtimerinfo001.obj
 0002:000028f0       $unwind$?NewObject@JNIEnv_@@QEAAPEAV_jobject@@PEAV_jclass@@PEAU_jmethodID@@ZZ 00000001800078f0     libtimerinfo001.obj
 0002:000028f0       $unwind$nsk_lcomplain      00000001800078f0     libtimerinfo001.obj
 0002:000028f0       $unwind$nsk_ldisplay       00000001800078f0     libtimerinfo001.obj
 0002:000028f8       $unwind$nsk_lvdisplay      00000001800078f8     libtimerinfo001.obj
 0002:000028f8       $unwind$_RTC_Initialize    00000001800078f8     MSVCRT:initsect.obj
 0002:000028f8       $unwind$_RTC_Terminate     00000001800078f8     MSVCRT:initsect.obj
 0002:000028f8       $unwind$?__scrt_initialize_thread_safe_statics@@YAHXZ 00000001800078f8     MSVCRT:thread_safe_statics.obj
 0002:00002904       $unwind$nsk_complain       0000000180007904     libtimerinfo001.obj
 0002:00002904       $unwind$nsk_printf         0000000180007904     libtimerinfo001.obj
 0002:0000290c       $unwind$nsk_lvcomplain     000000018000790c     libtimerinfo001.obj
 0002:00002924       $unwind$nsk_ltrace         0000000180007924     libtimerinfo001.obj
 0002:00002924       $unwind$__report_gsfailure 0000000180007924     MSVCRT:gs_report.obj
 0002:0000292c       $unwind$nsk_lvtrace        000000018000792c     libtimerinfo001.obj
 0002:0000292c       $unwind$__raise_securityfailure 000000018000792c     MSVCRT:gs_report.obj
 0002:0000292c       $unwind$__scrt_initialize_crt 000000018000792c     MSVCRT:utility.obj
 0002:0000292c       $unwind$__scrt_initialize_onexit_tables 000000018000792c     MSVCRT:utility.obj
 0002:0000292c       $unwind$__scrt_release_startup_lock 000000018000792c     MSVCRT:utility.obj
 0002:0000292c       $unwind$__scrt_uninitialize_crt 000000018000792c     MSVCRT:utility.obj
 0002:0000292c       $unwind$_onexit            000000018000792c     MSVCRT:utility.obj
 0002:00002934       $unwind$nsk_lverify        0000000180007934     libtimerinfo001.obj
 0002:00002944       $unwind$nsk_vprintf        0000000180007944     libtimerinfo001.obj
 0002:00002954       $unwind$?julong_to_string@@YAPEAD_KPEAD@Z 0000000180007954     libtimerinfo001.obj
 0002:00002964       $unwind$?nsk_jni_lverify@@YAHHPEAUJNIEnv_@@HQEBDH1ZZ 0000000180007964     libtimerinfo001.obj
 0002:00002978       $unwind$?nsk_jni_check_exception@@YAHPEAUJNIEnv_@@QEBDH@Z 0000000180007978     libtimerinfo001.obj
 0002:00002994       $unwind$nsk_jvmti_parseOptions 0000000180007994     libtimerinfo001.obj
 0002:000029b0       $unwind$nsk_jvmti_createJVMTIEnv 00000001800079b0     libtimerinfo001.obj
 0002:000029c4       $unwind$check_option       00000001800079c4     libtimerinfo001.obj
 0002:000029c4       $unwind$nsk_jvmti_waitForSync 00000001800079c4     libtimerinfo001.obj
 0002:000029c4       $unwind$_DllMainCRTStartup 00000001800079c4     MSVCRT:dll_dllmain.obj
 0002:000029d4       $unwind$Java_nsk_jvmti_unit_FollowReferences_FollowRefObjects_resetTags 00000001800079d4     libtimerinfo001.obj
 0002:000029d4       $unwind$addRefToVerify     00000001800079d4     libtimerinfo001.obj
 0002:000029d4       $unwind$nsk_jvmti_resetAgentData 00000001800079d4     libtimerinfo001.obj
 0002:000029d4       $unwind$nsk_jvmti_resumeSync 00000001800079d4     libtimerinfo001.obj
 0002:000029d4       $unwind$__scrt_initialize_default_local_stdio_options 00000001800079d4     MSVCRT:default_local_stdio_options.obj
 0002:000029d4       $unwind$?dllmain_crt_dispatch@@YAHQEAUHINSTANCE__@@KQEAX@Z 00000001800079d4     MSVCRT:dll_dllmain.obj
 0002:000029d4       $unwind$DllMain            00000001800079d4     MSVCRT:dll_dllmain_stub.obj
 0002:000029d4       $unwind$__GSHandlerCheck   00000001800079d4     MSVCRT:gshandler.obj
 0002:000029d4       $unwind$?__scrt_uninitialize_thread_safe_statics@@YAXXZ 00000001800079d4     MSVCRT:thread_safe_statics.obj
 0002:000029d4       $unwind$__scrt_acquire_startup_lock 00000001800079d4     MSVCRT:utility.obj
 0002:000029d4       $unwind$__scrt_dllmain_after_initialize_c 00000001800079d4     MSVCRT:utility.obj
 0002:000029d4       $unwind$__scrt_dllmain_before_initialize_c 00000001800079d4     MSVCRT:utility.obj
 0002:000029d4       $unwind$__scrt_dllmain_crt_thread_attach 00000001800079d4     MSVCRT:utility.obj
 0002:000029d4       $unwind$__scrt_dllmain_crt_thread_detach 00000001800079d4     MSVCRT:utility.obj
 0002:000029d4       $unwind$__scrt_dllmain_uninitialize_c 00000001800079d4     MSVCRT:utility.obj
 0002:000029d4       $unwind$__scrt_dllmain_uninitialize_critical 00000001800079d4     MSVCRT:utility.obj
 0002:000029d4       $unwind$atexit             00000001800079d4     MSVCRT:utility.obj
 0002:000029dc       $unwind$nsk_jvmti_enableEvents 00000001800079dc     libtimerinfo001.obj
 0002:000029f4       $unwind$nsk_jvmti_lverify  00000001800079f4     libtimerinfo001.obj
 0002:00002a08       $unwind$exitOnError        0000000180007a08     libtimerinfo001.obj
 0002:00002a18       $unwind$Java_nsk_share_jvmti_ArgumentHandler_getAgentOptionsString 0000000180007a18     libtimerinfo001.obj
 0002:00002a2c       $unwind$Java_nsk_jvmti_unit_FollowReferences_FollowRefObjects_getTag 0000000180007a2c     libtimerinfo001.obj
 0002:00002a2c       $unwind$Java_nsk_share_jvmti_DebugeeClass_checkStatus 0000000180007a2c     libtimerinfo001.obj
 0002:00002a2c       $unwind$agentThreadWrapper 0000000180007a2c     libtimerinfo001.obj
 0002:00002a3c       $unwind$startAgentThreadWrapper 0000000180007a3c     libtimerinfo001.obj
 0002:00002a58       $unwind$syncDebuggeeStatus 0000000180007a58     libtimerinfo001.obj
 0002:00002a58       $unwind$__scrt_dllmain_exception_filter 0000000180007a58     MSVCRT:utility.obj
 0002:00002a6c       $unwind$Java_nsk_share_jvmti_DebugeeClass_resetAgentData 0000000180007a6c     libtimerinfo001.obj
 0002:00002a74       $unwind$MA_checkStatus     0000000180007a74     libtimerinfo001.obj
 0002:00002a88       $unwind$Java_nsk_jvmti_unit_FollowReferences_FollowRefObjects_setTag 0000000180007a88     libtimerinfo001.obj
 0002:00002aa0       $unwind$Java_nsk_jvmti_unit_FollowReferences_FollowRefObjects_addRefToVerify 0000000180007aa0     libtimerinfo001.obj
 0002:00002abc       $unwind$Agent_Initialize   0000000180007abc     libtimerinfo001.obj
 0002:00002adc       $unwind$checkTimerInfo     0000000180007adc     libtimerinfo001.obj
 0002:00002afc       $unwind$agentProc          0000000180007afc     libtimerinfo001.obj
 0002:00002afc       $unwind$callbackVMInit     0000000180007afc     libtimerinfo001.obj
 0002:00002b0c       $unwind$callbackVMDeath    0000000180007b0c     libtimerinfo001.obj
 0002:00002b20       $unwind$capture_previous_context 0000000180007b20     MSVCRT:gs_report.obj
 0002:00002b2c       $unwind$__GSHandlerCheckCommon 0000000180007b2c     MSVCRT:gshandler.obj
 0002:00002b38       $xdatasym                  0000000180007b38     MSVCRT:amdsecgs.obj
 0002:00002b3c       $unwind$?dllmain_crt_process_attach@@YAHQEAUHINSTANCE__@@QEAX@Z 0000000180007b3c     MSVCRT:dll_dllmain.obj
 0002:00002b78       $unwind$?fin$0@?0??dllmain_crt_process_attach@@YAHQEAUHINSTANCE__@@QEAX@Z@4HA 0000000180007b78     MSVCRT:dll_dllmain.obj
 0002:00002b78       $unwind$?fin$0@?0??dllmain_crt_process_detach@@YAH_N@Z@4HA 0000000180007b78     MSVCRT:dll_dllmain.obj
 0002:00002b78       $unwind$?fin$1@?0??dllmain_crt_process_detach@@YAH_N@Z@4HA 0000000180007b78     MSVCRT:dll_dllmain.obj
 0002:00002b80       $unwind$?dllmain_crt_process_detach@@YAH_N@Z 0000000180007b80     MSVCRT:dll_dllmain.obj
 0002:00002bd4       $unwind$?dllmain_dispatch@@YAHQEAUHINSTANCE__@@KQEAX@Z 0000000180007bd4     MSVCRT:dll_dllmain.obj
 0002:00002bfc       $unwind$?filt$0@?0??dllmain_dispatch@@YAHQEAUHINSTANCE__@@KQEAX@Z@4HA 0000000180007bfc     MSVCRT:dll_dllmain.obj
 0002:00002c04       $unwind$__scrt_is_nonwritable_in_current_image 0000000180007c04     MSVCRT:utility.obj
 0002:00002c24       $unwind$__scrt_is_nonwritable_in_current_image$filt$0 0000000180007c24     MSVCRT:utility.obj
 0002:00002c2c       $unwind$__scrt_fastfail    0000000180007c2c     MSVCRT:utility_desktop.obj
 0002:00002c3c       $unwind$__security_init_cookie 0000000180007c3c     MSVCRT:gs_support.obj
 0002:00002c48       $unwind$__isa_available_init 0000000180007c48     MSVCRT:cpu_disp.obj
 0002:00002c58       $xdatasym                  0000000180007c58     MSVCRT:guard_dispatch.obj
 0002:00002c60       $xdatasym                  0000000180007c60     MSVCRT:guard_xfg_dispatch.obj
 0002:00002c70       .edata                     0000000180007c70     timerinfo001.exp
 0002:00002c98       rgpv                       0000000180007c98     timerinfo001.exp
 0002:00002cd8       rgszName                   0000000180007cd8     timerinfo001.exp
 0002:00002d18       rgwOrd                     0000000180007d18     timerinfo001.exp
 0002:00002d38       szName                     0000000180007d38     timerinfo001.exp
 0002:00002d49       $N00001                    0000000180007d49     timerinfo001.exp
 0002:00002d58       $N00002                    0000000180007d58     timerinfo001.exp
 0002:00002d65       $N00003                    0000000180007d65     timerinfo001.exp
 0002:00002daa       $N00004                    0000000180007daa     timerinfo001.exp
 0002:00002de7       $N00005                    0000000180007de7     timerinfo001.exp
 0002:00002e2f       $N00006                    0000000180007e2f     timerinfo001.exp
 0002:00002e6f       $N00007                    0000000180007e6f     timerinfo001.exp
 0002:00002eac       $N00008                    0000000180007eac     timerinfo001.exp
 0002:00002ee7       $N00009                    0000000180007ee7     timerinfo001.exp
 0002:00002f15       $N00010                    0000000180007f15     timerinfo001.exp
 0002:00002f46       $N00011                    0000000180007f46     timerinfo001.exp
 0002:00002f75       $N00012                    0000000180007f75     timerinfo001.exp
 0002:00002fa4       $N00013                    0000000180007fa4     timerinfo001.exp
 0002:00002fd9       $N00014                    0000000180007fd9     timerinfo001.exp
 0002:00002fe8       $N00015                    0000000180007fe8     timerinfo001.exp
 0002:00002ff8       $N00016                    0000000180007ff8     timerinfo001.exp
 0002:0000345a       .idata$6                   000000018000845a     kernel32:KERNEL32.dll
 0002:000034be       .idata$6                   00000001800084be     vcruntime:VCRUNTIME140.dll
 0002:00003650       .idata$6                   0000000180008650     ucrt:api-ms-win-crt-heap-l1-1-0.dll
 0002:00003670       .idata$6                   0000000180008670     ucrt:api-ms-win-crt-runtime-l1-1-0.dll
 0002:00003692       .idata$6                   0000000180008692     ucrt:api-ms-win-crt-convert-l1-1-0.dll
 0002:000036b4       .idata$6                   00000001800086b4     ucrt:api-ms-win-crt-stdio-l1-1-0.dll
 0002:000036d4       .idata$6                   00000001800086d4     ucrt:api-ms-win-crt-string-l1-1-0.dll
 0003:00000000       ?codeAttributeName@@3PEBDEB 0000000180009000     libtimerinfo001.obj
 0003:00000008       ?lineNumberAttributeName@@3PEBDEB 0000000180009008     libtimerinfo001.obj
 0003:00000010       ?localVarAttributeName@@3PEBDEB 0000000180009010     libtimerinfo001.obj
 0003:00000018       ?localVarTypeAttributeName@@3PEBDEB 0000000180009018     libtimerinfo001.obj
 0003:00000020       ?stackMapAttributeName@@3PEBDEB 0000000180009020     libtimerinfo001.obj
 0003:00000028       ?callBytes@@3PAEA          0000000180009028     libtimerinfo001.obj
 0003:0000002c       ?allocBytes@@3PAEA         000000018000902c     libtimerinfo001.obj
 0003:00000030       events                     0000000180009030     libtimerinfo001.obj
 0003:0001aad4       redefineAttempted          0000000180023ad4     libtimerinfo001.obj
 0003:0001aad8       nsk_context                0000000180023ad8     libtimerinfo001.obj
 0003:0001aae4       redefineSucceed            0000000180023ae4     libtimerinfo001.obj
 0003:0001aae8       agentFailed                0000000180023ae8     libtimerinfo001.obj
 0003:0001aaec       currentAgentStatus         0000000180023aec     libtimerinfo001.obj
 0003:0001aaf0       context                    0000000180023af0     libtimerinfo001.obj
 0003:0001aba8       agentThread                0000000180023ba8     libtimerinfo001.obj
 0003:0001abb0       agentThreadProc            0000000180023bb0     libtimerinfo001.obj
 0003:0001abb8       agentThreadArg             0000000180023bb8     libtimerinfo001.obj
 0003:0001abc0       agent_data                 0000000180023bc0     libtimerinfo001.obj
 0003:0001abd0       jvmti_env                  0000000180023bd0     libtimerinfo001.obj
 0003:0001abd8       jvm                        0000000180023bd8     libtimerinfo001.obj
 0003:0001abe0       jni_env                    0000000180023be0     libtimerinfo001.obj
 0003:0001abe8       checkStatus_func           0000000180023be8     libtimerinfo001.obj
 0003:0001abf0       ?codeAttributeIndex@@3GA   0000000180023bf0     libtimerinfo001.obj
 0003:0001abf4       ?lineNumberAttributeIndex@@3GA 0000000180023bf4     libtimerinfo001.obj
 0003:0001abf8       ?localVarAttributeIndex@@3GA 0000000180023bf8     libtimerinfo001.obj
 0003:0001abfc       ?localVarTypeAttributeIndex@@3GA 0000000180023bfc     libtimerinfo001.obj
 0003:0001ac00       ?stackMapAttributeIndex@@3GA 0000000180023c00     libtimerinfo001.obj
 0003:0001ac04       ?stackFrameOffset@@3GA     0000000180023c04     libtimerinfo001.obj
 0003:0001ac08       ?mode@@3HA                 0000000180023c08     libtimerinfo001.obj
 0003:0001ac0c       ?constantPoolSize@@3GA     0000000180023c0c     libtimerinfo001.obj
 0003:0001ac10       ?orig@@3PEBEEB             0000000180023c10     libtimerinfo001.obj
 0003:0001ac18       ?gen@@3PEAEEA              0000000180023c18     libtimerinfo001.obj
 0003:0001ac20       ?inputPos@@3PEAEEA         0000000180023c20     libtimerinfo001.obj
 0003:0001ac28       ?endPos@@3PEBEEB           0000000180023c28     libtimerinfo001.obj
 0003:0001ac30       ?genPos@@3PEAEEA           0000000180023c30     libtimerinfo001.obj
 0003:0001ac38       ?markPos@@3PEAEEA          0000000180023c38     libtimerinfo001.obj
 0003:0001ac40       ?constantPool@@3PEAPEADEA  0000000180023c40     libtimerinfo001.obj
 0003:0001ac48       ?constantPoolCount@@3GA    0000000180023c48     libtimerinfo001.obj
 0003:0001ac4c       ?zeroBytes@@3PAEA          0000000180023c4c     libtimerinfo001.obj
 0003:0001ac50       ?codeLength@@3IA           0000000180023c50     libtimerinfo001.obj
 0003:0001ac58       ?map@@3PEAIEA              0000000180023c58     libtimerinfo001.obj
 0003:0001ac60       ?widening@@3PEACEA         0000000180023c60     libtimerinfo001.obj
 0003:0001ac68       timeout                    0000000180023c68     libtimerinfo001.obj
 0003:0001ac70       initInfo                   0000000180023c70     libtimerinfo001.obj
 0003:0001aca0       GS_ExceptionRecord         0000000180023ca0     MSVCRT:gs_report.obj
 0003:0001ad40       GS_ContextRecord           0000000180023d40     MSVCRT:gs_report.obj
 0003:0001b210       ?g_tss_cv@@3U_RTL_CONDITION_VARIABLE@@A 0000000180024210     MSVCRT:thread_safe_statics.obj
 0003:0001b218       ?g_tss_event@@3PEAXEA      0000000180024218     MSVCRT:thread_safe_statics.obj
 0003:0001b220       ?g_tss_mutex@@3U_RTL_CRITICAL_SECTION@@A 0000000180024220     MSVCRT:thread_safe_statics.obj
 0003:0001b248       ?g_sleep_condition_variable_cs@@3P6AHPEAU_RTL_CONDITION_VARIABLE@@PEAU_RTL_CRITICAL_SECTION@@K@ZEA 0000000180024248     MSVCRT:thread_safe_statics.obj
 0003:0001b250       ?g_wake_all_condition_variable@@3P6AXPEAU_RTL_CONDITION_VARIABLE@@@ZEA 0000000180024250     MSVCRT:thread_safe_statics.obj
 0003:0001b25c       ?__proc_attached@@3HA      000000018002425c     MSVCRT:dll_dllmain.obj
 0003:0001b270       ?is_initialized_as_dll@@3_NA 0000000180024270     MSVCRT:utility.obj
 0003:0001b271       ?module_local_atexit_table_initialized@@3_NA 0000000180024271     MSVCRT:utility.obj
 0003:0001b278       ?module_local_atexit_table@@3U_onexit_table_t@@A 0000000180024278     MSVCRT:utility.obj
 0003:0001b290       ?module_local_at_quick_exit_table@@3U_onexit_table_t@@A 0000000180024290     MSVCRT:utility.obj
